:020000021000EC
:1000000041C0E4E7F9E200E000A301A302A303A3D7
:1000100004A305A3068907FF06C0048D158D012BD7
:1000200011F400E0089500918A29007631F40E94CD
:100030005D83002311F001E0089500918A290F717A
:0E004000013079F70E94B4810023A9F7EACFBE
:10007C000C94D6840C940E850091780005FDC9C0B3
:10008C00F092400608E1009356060FEF0A95002304
:10009C00E9F70091480606FFABC0E0E0F0E00791FD
:1000AC0016910F3F19F41F3F09F4A2C0B2C03BB721
:1000BC002BBFF8012091CA014093CA013DE930934E
:1000CC003400E8952093CA013BBF08953091CF01CD
:1000DC0037FDFCCF3BB72BBFF8012091CA0113E2CF
:1000EC001093CA010A01E8952093CA013BBF0895F9
:1000FC0027E402EA10E00E94FF800E946681789457
:10010C000E9481840E94B784FFCF00918C290F77C5
:10011C000093C304089500918C29002319F0025018
:10012C0039F005C024E030E004E111E218C041C010
:10013C0020E004EE10E250E032E0F0E0E22FEC516F
:10014C00FF4D40A1239FF801E00DF11D4283538325
:10015C0023952F3090F320E22093E42030E00E948E
:10016C00D08401E00895E4E7F9E2018D0A9529F0C5
:10017C000A95B9F00A95D1F01CC0E0ECF0E22289A6
:10018C0030E072968F010E94D084E4E7F9E2048D8E
:10019C00158D20A131A10217130710F400A311A390
:1001AC00E0CFE0ECF0E222813381ECCFB4DF00232E
:0601BC0061F700E0089568
:1001FC0007C040E04BBFF80158ED54BF2083089571
:10020C0001E70DBF00E20EBFC3E5DAE20E9456879C
:10021C006FDFF092560600910020109101200A3AEF
:10022C00154511F00C940000F0920020F092012082
:10023C0000E200937800F6CF4091CA01E22FF32F31
:10024C000093CA0104914093CA010895BA01A80110
:10025C00890102D1CBC261E06A93BA01A901FCD039
:10026C00D9C2B90198018B0154C20E942287D801CE
:10027C00C9012A0106C0FC012191CF018D015BD27D
:10028C00119682012FEF420E521E012BA1F7E6E0D0
:10029C000C942E8762E770E2260F371F0C94398777
:1002AC0066E271E2F9CFF8940AEA15E5E0E0F0E2D3
:1002BC000083118320917900216009E731D0FFCFB1
:1002CC0024E001E42DD02DE127D0009362002CE135
:1002DC0023D0009363001FB7F894E0E5F0E00081B1
:1002EC00026000831FBF0091510001FBE6F721E083
:1002FC0000E410E04AD2E6E5F0E00081097F0083DB
:10030C0000E807870BEB008B008104600083E0E6BC
:10031C00008101600083089530E002E00C9422819A
:10032C0010E033C200E00093302159D000919000CE
:10033C0000932621009191000093272100919200B7
:10034C000093282100919300009329210091D00162
:10035C0001FB16F001E001C000E0D7C07ED4AAE892
:10036C00B9E200918A2900760032B9F510918B29F7
:10037C000C91569707FF15C0125049F01A9551F57C
:10038C0026E030E000E211E285D001E027C0C1D0C8
:10039C000289138920E000301207E1F0F801099579
:1003AC001DC01A9521F01350A9F419D0EECF00916D
:1003BC003021002331F009E511E892960D931C933E
:1003CC00E4CF20E430E003E311E264D00FEF11E856
:1003DC009496F4CF9ED00FE076D000E03BC400C0E2
:1003EC0000E0B8D093D100E004A305A302A303A3BB
:1003FC000895F5DF10E08DD0128B138BE3E3F1E25F
:10040C0030812181203001E0300709F428C02030F0
:10041C0003E0300709F43FC02130300709F457C01E
:10042C00203004E0300761F40091CF0107FDFCCFD0
:10043C0040E200E011D00E945D80C9D100E065C0AF
:10044C002330300721F401E000933021089523304C
:10045C00364009F44BC0AEC020E030E0089559D0CE
:10046C00018D128D012309F072C026813781203055
:10047C00304011F427D002C020D009F49BC020E0FA
:10048C0038E006D007E413E841D104A315A33FC01C
:10049C0004E711E27FC211D019F021D011F412D06F
:1004AC0089C0018D128D012319F00DEA12E802C0EA
:1004BC0002EE12E8028B138B2AC005E311E250D036
:1004CC000023089503E000870AE004870895F5DF10
:1004DC0019F005D011F4F6DF6DC080D018C0E8E13A
:1004EC00F1E224813581203030400895E3E3F1E2DC
:1004FC000281002349F40381013108F055C00CD06E
:10050C0000E007D0048B058B02C00093312101E081
:10051C000895E8E1F1E20895033041F0023031F042
:10052C00043021F0053011F011E001C010E01093FF
:10053C00322112E0019FF001E356FF4D6081F18101
:10054C0008E111E2E62F48E050E00C94128703E03A
:10055C0001D030C00093202102E0009324210895A3
:10056C00BD01F80150810181402FACE2B1E20D9345
:10057C005C935597128130E0038120E00D901D9023
:10058C002D903C901397001511052205330510F0A2
:10059C000BD008C0041B150B0F5F1F4FFD01068B02
:1005AC00178B01E0DB01089508E0009320210AE09D
:1005BC000093242100E0089550D3A8E1B1E2FD019D
:1005CC00468957894ED01496ED91FC911597099553
:1005DC00FD01268937895CDF01E03CC3C2D0A8E16C
:1005EC00B1E2FD0106891789012B39F400E018EFFF
:1005FC00068B178B80E098E010C0FD0106891789E7
:10060C00202F212B59F1183010F4C80102C080E0C2
:10061C0098E0081B190B068B178BAC0122D0648158
:10062C00F581E62F099504E711E207C0FD01248945
:10063C0035892F5F3F4F248B358B9C010197232BE2
:10064C00E1F2F80121918F012F3F81F305E0009336
:10065C0020210CE313E8FD01028B138BE4E00C94D6
:10066C0030872489358904E711E2089552DF248903
:10067C000589009374212093752122E030E008DF76
:10068C0046CF47DF0489158946895789202F2F7358
:10069C00622F70E024E731E2260F371F6681F78165
:1006AC00E62F099500E032D004A305A330CF2ED05D
:1006BC0006890F7109F07ECF1789068907FF13C0D1
:1006CC00112329F0165039F0125039F0F4CF22E0F2
:1006DC0030E0B69605C00C94B98021E030E0BC96B1
:1006EC008F01D8DE14CF155019F0145031F0E3CF30
:1006FC000BE810E802A313A3F5CF01E010E006A36A
:10070C0017A3008D04A7002369F30CCEE4E7F9E2EC
:10071C000895B90132D0208127FDFDCFECEC20816A
:10072C0028602083105F98018B01B8DDECECF1E0C0
:10073C000081077FEFCD15D0C801A22FB091CA015F
:10074C0012D01BD0008107FDFDCF3AD09093C10190
:10075C008093C001A093C40105E312D0B093CA01E9
:10076C007DCF0C94248709D0008107FDFDCF00813B
:10077C0001FF02C006E304D00895EFECF1E0089508
:10078C000093CA0121E00BEC11E00C94FF809A93CA
:10079C008A93802F9091CA01E6DF0091CF0107FD6B
:1007AC00FCCF0ED00093C1010093C0018093C40113
:1007BC0003950032C8F39093CA01899199910895D9
:1007CC0003E30093CA0100E00093C20108958A93E9
:1007DC000FEFDDDFD2DF008107FDFDCF8091CA0175
:1007EC0000E3CEDF8093CA01899108952091CF0157
:1007FC0027FDFCCF262F272B61F0F80130E03BBF03
:10080C002691FA012193AF010F5F1F4F6150704089
:10081C00F1CF08950E941D8722974A012B016D8408
:10082C00D801912F80E007C04091CF0147FDFCCF4C
:10083C0045E20E945D80042D052909F442C0AA24DA
:10084C000091CF0107FDFCCF00E8702E662071F0FF
:10085C00FC0130E03BBF0791169108831983088196
:10086C000F3F1F4F31F0AA24A39403C00FEF08834E
:10087C000983042D052979F0A817B90729F425D087
:10088C000883042D052939F0FC013196AE17BF07FA
:10089C0011F41BD00983488159818C01DDDD0E9444
:1008AC006C8002967A9491F6AC015A95AA208A0132
:1008BC00D3DD09F0B9CF4091CF0147FDFCCF44E225
:1008CC00B8CF2296ECE00C9429870FEF400E501E07
:1008DC001196F40101914F0108952AE107D000937C
:1008EC00FA042BE103D00093FB04089515DD0F3FB0
:1008FC0009F40FE108950E94258700E00093600041
:10090C0023E004E40DDD67D20064008301E0009372
:10091C0060000FB7F894A02F9FDD8901E3D0F80198
:10092C00EC58F64D358323952230B8F3D6DF009181
:10093C00C0040093C0044FD20068008300810061A2
:10094C00008384E799E20496E6EC80839183E0ECE3
:10095C002FD10FEF0583E8ECDBDCAFBFE3E00C94A9
:10096C0031871FB7F89400E43AD200E238D2E1ECB8
:10097C00F4E0CEDCE9EC008102600083E8EC00815D
:10098C0000640083E9ECC4DCE8EC008100680083BF
:10099C001FBF0895BBDE068F178F20A331A30895C8
:1009AC0065D00091CB0407FF02C000E82EC0FCD13B
:1009BC00002361F5EBEC10D204FF1EC000E10FD256
:1009CC0000E00093A02901E010E000939A29109315
:1009DC009B2900E00093C30420E430E05AD020E4CB
:1009EC0030E010E000E855D003EA19E200937C29CE
:1009FC0010937D292ED10AC0008106FF02C000E4AD
:100A0C0004C0008105FF02C000E2E9D11CD018959A
:100A1C002DD0E8D10023B1F402E00093CC04009176
:100A2C00C50422D0F801008105FF06C01DD020E2CC
:100A3C00F801269315D106C000E817D020E2F80182
:100A4C002693B9D0E3CF9BBF8FBF09911991299100
:100A5C0039914991599169917991099019902990FD
:100A6C003990E991F991A9CE00E02DC09A938A931F
:100A7C00FA93EA933A922A921A920A927A936A9386
:100A8C005A934A933A932A931A930A938FB79BB724
:100A9C0008958A932051304041F02051304039F074
:100AAC002052304031F080E005C081E003C082E08C
:100ABC0001C083E0DADF20E0F801218326E0208307
:100ACC008064818391CE68E779E2202F2F70220F0A
:100ADC00402F440F00E010E0001F020F03D0060F60
:100AEC00171F089543E00C940C879D01E8EC74D11A
:100AFC000F7D008300810F7D00833FD102E00593C1
:100B0C00A2E8B9E200E010E00D930C93539600E2DA
:100B1C00069300E406933BD1069300E406931D93E1
:100B2C001D931D931C9315971D931C9311A7D9010D
:100B3C0008950CD1002331F0033011F0043009F486
:100B4C0029D187D0E3DD06811781083050E01040B1
:100B5C0039F548E023EA39E20AE819E29FDBE8ECD0
:100B6C00F4E026D025D00E940180002309F4F1C0C6
:100B7C00CDDD068907FF0BC000A10F7311F401E056
:100B8C0001C000E006A70ED002E005A714C0048D3A
:100B9C00158D012B09F405C005D001E005A7F3D094
:100BAC000895E3C000E000A701A702A703A70895DA
:100BBC0000810062AFCB51D0C7D0033011F448D0C4
:100BCC0046C0FD0120A131A142A553A58901041BFA
:100BDC00150B402F412B21F506A5002311F4D0D085
:100BEC0036C000A511A5020F131F248D358D0217D9
:100BFC00130728F089D019F00995002339F400E087
:100C0C000093A229FD01068707871FC070D020A181
:100C1C0011A1022F2F7311F421E001C020E026A7AF
:100C2C00013420E0120710F000E410E0068717876B
:100C3C00268D378D42A553A5240F351F208B318B64
:100C4C009A01200F311F22A733A797D09DD002C045
:100C5C00A1D04BCFA991B9910895BA93AA930895B5
:100C6C0080DD72D0043011F4F3DF40C0FD018681C9
:100C7C00978162A573A520A131A18B01080F191FC3
:100C8C002017310718F4C901861B970BAC0123EA16
:100C9C0039E2068D178D060F171F00DBFD0102A52B
:100CAC0013A5080F191F02A713A78034904031F425
:100CBC0026D0448D558D2417350760F000A311A361
:100CCC0094966FD029F00995002311F442D00EC0F0
:100CDC004CD00CC020A131A12017310731F414D015
:100CEC00A9F30995002391F302D04DD0B7CCFD01A7
:100CFC0002A513A504D020A731A700E056CF20A54C
:100D0C0031A5200F311F08959496ED91FC91959784
:100D1C0000E0E030F00708950091782905FD07C048
:100D2C0015D0013009F43DCF043009F415D00895E5
:100D3C000091802905FD07C009D0023009F420C0BC
:100D4C00033009F409D00895A4E7B9E20091A12970
:100D5C00089505E00093A129E1E8F9E204E0059388
:100D6C00E9E7F9E204E005930895D0DC03E005A778
:100D7C0000E00687078701D007C0E0E8F9E2089594
:100D8C0004E00093A12903D002E006930895E8E75C
:100D9C00F9E2089562DFA6E9B9E203D009F00995FA
:100DAC0059CFED91FC91B4CFEBEC16D002FF07C0FC
:100DBC00F093CA040091802906FDAEDFA8CB008118
:100DCC0001FF08C002E00BD00091782906FFF6CF96
:100DDC00AFDFF4CFEFCBE0ECF4E0008108950093AB
:100DEC00CA0408950091CC0400FFE4CB01E0009309
:100DFC00CC04CDDF00E80693C0DF00E8069301E0E9
:100E0C00EEDFC5DF00E1069394DE81CB4A951AF044
:100E1C00000F111FFBCF0895AF93BF93D801019022
:100E2C000D9241505040D9F7BF91AF910895AA92BD
:100E3C009A928A927A926A925A924A92BA93AA9304
:100E4C009A938A930895AA84998488847F806E806B
:100E5C005D804C80BB81AA8199818881F0E0EC0F88
:100E6C00FD1FEF010895BD01D801F90104C02191C6
:100E7C002D9341505040242F252BC9F7DB010895A9
:100E8C0020E008D0E9F708953BBF27913BB702D08B
:100E9C00D9F708952D9301501040202F212B089540
:100EAC000CE0402E0FE0502E01E0602EF201362DAA
:100EBC006BBE07911691F201EE5FFF4F3F4F3BBFA8
:100ECC00A791B691F201362DEC5FFF4F3F4F3BBF20
:100EDC00479157916691242F252B262B21F0FA014F
:100EEC00362FD2DF01C0CCDF07E0400E00E0501EF1
:100EFC00601EA201662D4A315F406140B8F2089530
:100F0C00CB081821000000A60072201A0F01030064
:100F1C0000000001002C8131810008000037813B6A
:100F2C008103000000508100000400000056810085
:100F3C0000000000000000000075207D2095209529
:100F4C002085208D20952095209520952095209505
:100F5C0020952095209520952095200009021200BF
:100F6C00010100C0320904000000FF000000120162
:100F7C00000200000040EB03E12F0300000200011F
:100F8C000003000000000000000000000000000052
:100F9C000000000000000000000000000000000045
:100FAC00444655204154584D454741363442310052
:040FBC00040309041D
:0400000310000000E9
:00000001FF
